:10000000E1C00000FCC00000FAC00000F8C0000021
:10001000F6C00000F4C00000F2C00000F0C0000014
:10002000EEC00000ECC000000C94C10AE8C0000063
:10003000E6C00000E4C00000E2C00000E0C0000034
:10004000DEC00000DCC00000DAC00000D8C0000044
:10005000D6C00000D4C00000D2C00000D0C0000054
:10006000CEC00000CCC00000CAC00000C8C0000064
:10007000C6C00000C4C00000C2C00000C0C0000074
:10008000BEC00000BCC00000BAC00000B8C0000084
:10009000B6C00000B4C00000B2C00000B0C0000094
:1000A000AEC00000ACC00000AAC0000005010905F8
:1000B000A10115002501350045017501950D0509C2
:1000C0001901290D81029503810105012507463B90
:1000D0000175049501651409398142650095018116
:1000E0000126FF0046FF0009300931093209357544
:1000F00008950481020600FF09200921092209232D
:10010000092409250926092709280929092A092B6B
:10011000950C81020A21269508B1020A2126910236
:1001200026FF0346FF03092C092D092E092F751000
:1001300095048102C01201100100000040100082ED
:10014000000100010200011201100100000040C482
:1001500010C0820100010200010902290001010012
:1001600080FA0904000002030000000921110100C7
:1001700001228900070502034000010705810340B1
:10018000000104030904200341006B0069007300AF
:1001900068006F0070002000430075007300740059
:1001A0006F006D00730000001A035000530033000D
:1001B000360030002B002000760031002E00300089
:1001C0003000000011241FBECFEFDAE0DEBFCDBF4C
:1001D00011E0A0E0B1E0E6E2FDE102C005900D9281
:1001E000A431B107D9F711E0A4E1B1E001C01D923B
:1001F000A134B107E1F70E9419090C94910E00CFC8
:10020000CF92DF92EF92FF920F931F93CF93DF93E2
:100210002FB12095237369B153B150955077FC01EC
:1002200088E08283178211861286108610821182DE
:100230001586138616861486128A118A108A1786E6
:1002400080E88383848385838683148A138A168A4D
:10025000158A108E178A128E118E80912B0130E034
:10026000882349F121FF03C010922C011CC024FFF8
:1002700002C081E003C025FF04C082E080932C010E
:1002800012C020FF10C080910B01882361F0809183
:100290002A01882321F481E080932A0102C0109270
:1002A0002A0110920B0154FF56C110922B0181E0DC
:1002B00080930B0150C121FF33C080912C01882312
:1002C000B9F4C9018072907024FF07C0892B61F4D2
:1002D00087E082838FEF87836EC0892B29F081E0CE
:1002E00082838FEF87837EC012828FEF878385C0E2
:1002F000813051F41482C9018072907024FD37C09E
:10030000892B09F47AC072C0823051F41682C90177
:100310008072907024FD3DC0892B09F46EC06BC0C3
:1003200020FF3EC080912C018823C1F4C901807256
:10033000907024FF07C0892B61F485E082838FEFE2
:10034000818739C0892B29F083E082838FEF8187F1
:1003500049C084E082838FEF81874FC0813081F470
:100360004FEF4483C9018072907024FF04C0892B31
:1003700009F043C026C0892B09F43FC043833DC028
:10038000823071F44FEF4683C9018072907024FF70
:1003900003C0892B91F51BC0892B79F145832DC0B2
:1003A00024FF17C080912C01882339F425FD25C036
:1003B00086E082838FEF828720C0813021F425FD83
:1003C0001CC013821AC0823021F425FD16C015828C
:1003D00014C025FF12C080912C01882329F482E0EB
:1003E00082838FEF808709C0813019F48FEF838378
:1003F00004C0823011F48FEF8583962F9095292FBA
:1004000030E041E0C42ED12CC222D32290FF05C09F
:100410008081816080838FEF828B82E0E82EF12CD7
:10042000E222F32221FF05C08081886080838FEF64
:10043000878789010470107022FF05C08081806267
:1004400080838FEF868723FF05C080818061808352
:100450008FEF8587E901C071D07024FF05C08081CE
:10046000826080838FEF818BB9016072707025FF8D
:1004700005C08081846080838FEF808BD901A07458
:10048000B07026FF05C08081806880838FEF8487ED
:1004900097FF05C08081806480838FEF8387452F1D
:1004A00050E09A012071307044FF03C08181826066
:1004B000818345FF44C0CC2041F0EF2831F0012B6F
:1004C00021F081E080932B011EC0CD2B69F0672BBA
:1004D000D1F010821586138616861486128A118A28
:1004E000108A178684E011C0672B69F0AB2B59F096
:1004F00010821586138616861486128A118A108A2F
:10050000178688E002C0818181608183232BB9F046
:1005100020912D0130912E0181E02C32380740F0DE
:1005200080912A01882321F48181806181830BC01D
:100530002F5F3F4F30932E0120932D0104C0109266
:100540002E0110922D0146FF06C0818180618183BA
:1005500081E080932A01DF91CF911F910F91FF904D
:10056000EF90DF90CF90089584B1807784B985B102
:10057000876085B9239A1CBC8CB580648CBD8CB512
:1005800080628CBD8CB588608CBD8CB584608CBD60
:100590002F9827980895982F27988DB581118EB59B
:1005A0009EBD90E025E008C0822F8A95F1F79F5FFD
:1005B000993C11F48AEA08950DB407FEF5CF611154
:1005C000279A8EB508952F923F924F925F926F9225
:1005D0007F928F929F92AF92BF92CF92DF92EF92D3
:1005E000FF920F931F93CF93DF93882E81E090E0CB
:1005F00020E80FB6F89420936100809361000FBE4D
:10060000B3DF00E0BB24BA9480E8982E15E3612E96
:10061000B3E77B2EA9E75A2EF1E44F2EECEF3E2EE6
:100620007BEF272E2798BEBC1899FCCF9FB19095E1
:100630009373A9B0A09413B110951077B0920101F3
:10064000B0920201909203019092040190920501F0
:100650009092060110921401109215011092160149
:1006600010921701109218011092190110921A019C
:1006700010921B0110921C0110921D0110921E017C
:1006800010921F0180912B01492F50E0882349F1DE
:1006900091FF03C010922C011CC094FF02C081E0A6
:1006A00003C095FF04C082E080932C0112C090FF2C
:1006B00010C080910B01882361F080912A0188236A
:1006C00021F481E080932A0102C010922A01109245
:1006D0000B0114FFBDC110922B0181E080930B012F
:1006E000B7C191FF22C080912C018823A1F48FEE25
:1006F00080930101B09216019A012072307094FF2C
:1007000005C0232B09F087C08FE65DC0232B09F4B9
:1007100082C08FEC74C0813019F4109204012CC097
:10072000823019F41092060138C040FF41C0809118
:100730002C018823E9F490910101892F8F7B80930C
:100740000101B09217019A012072307044FF07C076
:10075000232B09F060C09F739093010136C0232BB7
:1007600009F459C09F7990930101B092140153C0CC
:10077000813079F4B09204019A012072307044FF04
:1007800004C0232B09F047C027C0232B09F443C022
:100790003BC0823069F4B09206019A012072307039
:1007A00044FF03C0232BB9F51EC0232BA1F131C098
:1007B00044FF1CC080912C01882351F445FD2BC0BF
:1007C000809101018F7780930101B092150123C0C0
:1007D000813029F445FD1FC0109203011CC08230F6
:1007E00029F445FD18C01092050115C045FF13C03E
:1007F00080912C01882331F4809101018F7D8093B9
:100800000101B3CF813019F4B092030104C08230EA
:1008100011F4B09205012A2D30E061E0C62ED12CF2
:10082000C222D322A0FE05C08FE780930201B092BE
:10083000190152E0E52EF12CE222F32221FF07C03C
:10084000809102018F7E80930201B0921801E9012C
:10085000C470D07022FF07C080910201877F80930F
:100860000201B0921D0123FF07C0809102018B7F1E
:1008700080930201B0921C01D901A071B07024FFD5
:1008800007C0809102018F7B80930201B0921A0110
:10089000B9016072707025FF07C0809102018F7DE1
:1008A00080930201B0921B01F901E074F07026FF01
:1008B00007C0809102018D7F80930201B0921F01D9
:1008C000A7FE07C0809102018E7F80930201B09243
:1008D0001E01412F50E09A012071307014FF05C0B5
:1008E00080910101877F8093010145FFA2C0CC2048
:1008F00041F0EF2831F0CD2B21F081E080932B01E6
:1009000052C0AB2B39F1672B09F44DC0B0920201F4
:100910009092030190920401909205019092060139
:1009200010921401109215011092160110921701E5
:10093000109218011092190110921A0110921B01C5
:1009400010921C0110921D0110921E0110921F01A5
:100950008DEF2CC0672B39F1EF2B29F1B0920201FA
:1009600090920301909204019092050190920601E9
:100970001092140110921501109216011092170195
:10098000109218011092190110921A0110921B0175
:1009900010921C0110921D0110921E0110921F0155
:1009A0002092010147C2809101018E7F8093010155
:1009B00041C220912D0130912E012F30310590F14F
:1009C00080912A01882371F583E0881659F580917A
:1009D00000018823A9F1B092020190920301909244
:1009E0000401909205019092060110921401109258
:1009F0001501109216011092170110921801109211
:100A0000190110921A0110921B0110921C011092F0
:100A10001D0110921E0110921F01309201011092CF
:100A200000010EC02F5F3F4F30932E0120932D0108
:100A300007C010922E0110922D0181E080930001D9
:100A400046FF06C083E0881619F481E080932A01EE
:100A50008FEF61E0A0DDF82E81E0F81609F0E2C129
:100A600080912001882309F418C183EF61E093DDB0
:100A7000182F8AE561E08FDD163409F48FC0173432
:100A800090F4133409F43FC0143430F41034D9F026
:100A9000113409F0C7C120C0143409F44DC0153415
:100AA00009F0C0C168C01C3409F4A5C01D3420F48D
:100AB000173409F0B7C194C01D3409F4BDC01F3408
:100AC00009F0B0C1D6C080E061E065DD082F80E0AC
:100AD00061E061DD82E0D7C080912101813041F485
:100AE0008FEF61E058DD8FEF61E055DD83E0CBC033
:100AF00080E061E050DD80E061E04DDD80E061E0BC
:100B00004ADD80E090C080E061E045DD082F80E0B4
:100B100061E041DD80E061E03EDD80E061E03BDD01
:100B200080E061E038DD80E060E035DD002309F041
:100B300079C11092200176C180E061E02CDD082FA0
:100B400080E061E028DD80E061E025DD80E061E0BB
:100B500022DD80E061E01FDD80E060E01CDD01302F
:100B600029F470920701009321015CC140920701B2
:100B70001092210157C183E061E00DDD082F82E072
:100B800061E009DD80912101813009F080E061E0C0
:100B900002DD82E061E0FFDC81E048C080E061E0EE
:100BA000FADC082F882359F480E061E0F4DC81E06E
:100BB00061E0F1DC82E061E0EEDC80E00DC08130DC
:100BC00009F030C180E061E0E6DC81E061E0E3DC77
:100BD00081E061E0E0DC81E061E0DDDC8FE029C004
:100BE00080E061E0D8DC80E061E0D5DC82E061E0BB
:100BF000D2DC80E0CFCF80E061E0CDDC082F88231D
:100C000041F480E061E0C7DC80E061E0C4DC84E0C6
:100C10000AC0813009F006C180E061E0BCDC80E000
:100C200061E0B9DC87E061E0B6DC80E061E0B3DC84
:100C300080E060E0B0DCF6C08091080161E0ABDCF0
:100C4000809308018091090161E0A5DC809309018E
:100C50008FEF61E0A0DC8FEF61E09DDC8FEF61E062
:100C60009ADC8FEF60E097DC70920701F09221012F
:100C7000D9C05092070180E061E08DDC082F80E050
:100C800061E089DC80E061E086DC80E061E083DCBB
:100C900080E061E080DC8AE5CCCF8091070161E0F3
:100CA0007ADC182F8AE561E076DC809107018134D7
:100CB00049F48091010161E06EDC082F809102010E
:100CC00060E069DC80910701833759F5809101016B
:100CD00061E061DC082F8A3A09F4A4C08091020126
:100CE00061E059DC8A3A09F49DC08091050161E018
:100CF00052DC8A3A09F496C08091060161E04BDC2F
:100D00008A3A09F48FC08091030161E044DC8A3A99
:100D100009F488C08091040160E03DDC8A3A09F45E
:100D200081C080910701893709F076C08091010167
:100D300061E031DC082F8A3A09F474C08091020125
:100D400061E029DC8A3A09F46DC08091050161E017
:100D500022DC8A3A09F466C08091060161E01BDC5E
:100D60008A3A09F45FC08091030161E014DC8A3A99
:100D700009F458C08091040161E00DDC8A3A09F45D
:100D800051C08091140161E006DC8A3A09F44AC03E
:100D90008091150161E0FFDB8A3A09F443C080913C
:100DA000160161E0F8DB8A3A09F43CC08091170132
:100DB00061E0F1DB8A3AB1F18091180161E0EBDB8F
:100DC0008A3A81F180911B0161E0E5DB8A3A51F1B9
:100DD00080911A0161E0DFDB8A3A21F180911901EB
:100DE00061E0D9DB8A3AF1F080911C0161E0D3DB4C
:100DF0008A3AC1F080911D0161E0CDDB8A3A91F021
:100E000080911E0161E0C7DB8A3A61F080911F0189
:100E100060E0C1DB8A3A31F0133421F4013011F47F
:100E200000932001279803C0862D8A95F1F7189921
:100E3000F9CBFACF232B09F4FCCDBBCD84B7877F48
:100E400084BF88E10FB6F894809360001092600030
:100E50000FBE81E090E020E80FB6F8942093610087
:100E6000809361000FBE84B1807784B985B18660BC
:100E700085B985B1867085B988B18F7388B981B31A
:100E80008F7381BB87B18F7387B980B38F7380BB3A
:100E9000729A76986A9A6E9A80B38C7C80BB81B382
:100EA000836381BB8AB11AB88BB18FEF8BB984B1E0
:100EB0008F7884B985B1806785B9089508950895BC
:100EC00081E0809325010895109225010895EF9205
:100ED000FF920F931F93DF93CF93CDB7DEB76B973E
:100EE0000FB6F894DEBF0FBECDBFEDB6FEB6809153
:100EF0003A01853009F495C0863020F4813009F03C
:100F0000DAC007C0863009F455C0893009F0D3C073
:100F10009FC080913901813A09F0CDC080913B0199
:100F200090913C018050934089F50DB71EB7809198
:100F30003F01909140012DB73EB7281B390B0FB6EA
:100F4000F8943EBF0FBE2DBF8DB79EB70196AC0182
:100F5000DC01ECE0F1E088E001900D928150E1F7D6
:100F60008091E800877F8093E80060913F01709155
:100F70004001CA0151D58091E8008B778093E80049
:100F80000FB6F8941EBF0FBE0DBF95C08E010F5F48
:100F90001F4FC80135D98091E800877F8093E80012
:100FA000C8016BE170E038D58091E8008B778093C1
:100FB000E80081C080913901803809F07CC020911F
:100FC0003B0130913C01432F809133018F5F80932F
:100FD00033012050314099F480913F0190914001BC
:100FE0008830910511F0429751F480912F018F5F65
:100FF00080932F01809130018F5F809330014230C8
:1010000049F480913F01909140018055914009F051
:1010100052C018C0433009F04EC081E080933101C6
:101020004AC080913901882309F045C0809133017D
:10103000882319F481E0809332018091300181305E
:1010400009F039C080912F018F5F80932F0133C049
:1010500080913901882379F580913101882329F421
:1010600080912F018F5F80932F0180912F01843019
:1010700010F1809124018823F1F4F8948091E0002C
:1010800081608093E00009D280E49CE90197F1F748
:1010900010922F011092300172986E988CE291E0BC
:1010A00020E931E0F9013197F1F70197D9F783E0B1
:1010B00080930A0188DA0FB6F894FEBE0FBEEDBE2B
:1010C0006B960FB6F894DEBF0FBECDBFCF91DF9108
:1010D0001F910F91FF90EF90089581E061EC42E342
:1010E00054D182E060EC42E350C10F931F93DF9331
:1010F000CF93CDB7DEB76B970FB6F894DEBF0FBEB8
:10110000CDBF80913801843009F04BC082E08093DC
:10111000E9008091E80082FF2DC08091E80085FF02
:1011200024C0CE01019668E070E040E050E042D576
:101130003E983F98869887988B81813059F082300D
:1011400071F0843089F0883011F4879A0EC08930AC
:1011500019F4879A3E9A09C08A3019F4879A3F9AFF
:1011600004C08C3011F4879A869A8091E8008B77BE
:101170008093E80081E08093E9008091E80080FF9F
:1011800010C08E010F5F1F4FC8013AD8C8016BE134
:1011900070E040E050E060D58091E8008E77809369
:1011A000E8006B960FB6F894DEBF0FBECDBFCF91AF
:1011B000DF911F910F91089580E090E020E80FB635
:1011C000F89420936100809361000FBEC2D178949F
:1011D00080912501882311F18091260190912701AA
:1011E000A0912801B091290180342DE0920723E0DD
:1011F000A20720E0B20760F40196A11DB11D809303
:10120000260190932701A0932801B09329010EC0D5
:1012100083B18095807551F0A1D008C0109226014D
:101220001092270110922801109229015EDF66D5E5
:10123000CFCF04DE80E49CE90197F1F789B1809576
:1012400080FF08C081E08093240120E030E040E08E
:1012500050E01DC081FF12C072986E988CE291E040
:1012600020E931E0F9013197F1F70197D9F781E0F1
:101270008093240183E080930A0107C084FFE5CFB7
:1012800081E08093240180910A019DD9DECF199BD2
:1012900006C083B190E083709070892B39F48091FF
:1012A0000A0191D920E030E040E050E02F5F3F4F4D
:1012B0004F4F5F4F203E83E9380784E0480780E0C6
:1012C000580728F379DF80E090E00895DA01933041
:1012D000F1F0943030F4913071F0923009F036C072
:1012E00005C0913249F1923289F52BC0E9E5F1E070
:1012F00029E230E02FC080913201882319F4E5E320
:10130000F1E002C0E7E4F1E022E130E023C0813007
:1013100049F0813018F08230C9F40AC0E2E8F1E007
:10132000849103C0E6E8F1E08491282F30E012C0F8
:10133000E8EAF1E08491F9CFEBE6F1E029E030E072
:1013400009C0ECEAF0E029E830E004C0E0E0F0E0B9
:1013500020E030E0ED93FC93C901089580E189BD60
:1013600089B5826089BD09B400FEFDCF8091D800A7
:101370008F7D8093D8008091E00082608093E000B0
:101380008091E00081FDFCCF0895382F282F2CC0DC
:101390002093E900231721F4762F942F50E006C004
:1013A0007091EC009091ED005091F00091FF1BC006
:1013B0008091EB008E7F8093EB008091ED00827036
:1013C0008093ED008091EB0081608093EB0070933F
:1013D000EC009093ED005093F0008091EE0087FDBB
:1013E00002C080E008952F5F273090F23093E9002B
:1013F00081E008958091390188239CF404C0809194
:1014000038018823B9F08091E80082FFF8CF8091FD
:10141000E8008B778093E800089580913801882355
:1014200049F08091E80080FFF8CF8091E8008E7746
:101430008093E80008954091E4005091E50024E68F
:101440008091EC0080FF05C08091E80080FF05C01E
:1014500022C08091E80082FD1EC08091380188235F
:1014600011F482E00895853011F483E008958091AD
:10147000EB0085FF02C081E008958091E400909127
:10148000E50084179507E1F2222311F484E0089522
:101490002150AC01D5CF80E0089566D06DD0E0EE4C
:1014A000F0E0808181608083A8EDB0E08C918F773F
:1014B0008C9319BCE7EDF0E080818E7F80838C9166
:1014C0008F7E8C93109237010895EF92FF920F93C5
:1014D0001F934AD051D008ED10E0F8018081982F79
:1014E0009F7790838068808380818F7D808319BC03
:1014F0001092380110923601109235011092340189
:1015000080EEE82EF12CF70180818B7F8083F8013B
:1015100080818160808380E060E042E336DFE1EE3D
:10152000F0E080818E7F8083E2EEF0E08081816058
:101530008083808188608083F70180818E7F8083B3
:10154000F8018081806180831F910F91FF90EF905F
:101550000895E7EDF0E08081816080838AE482BFB6
:1015600081E080933701B1CFE8EDF0E080818E7F9C
:1015700080831092E20008951092DA001092E10048
:1015800008951F920F920FB60F9211242F933F933D
:101590004F935F936F937F938F939F93AF93BF937B
:1015A000EF93FF938091E10082FF0AC08091E200F7
:1015B00082FF06C08091E1008B7F8093E1002BD2F7
:1015C0008091DA0080FF1EC08091D80080FF1AC091
:1015D0008091DA008E7F8093DA008091D90080FFBD
:1015E0000DC080E189BD89B5826089BD09B400FE66
:1015F000FDCF81E08093380161DC04C019BC1092FA
:1016000038015DDC8091E10080FF18C08091E2002C
:1016100080FF14C08091E2008E7F8093E200809171
:10162000E20080618093E2008091D8008062809324
:10163000D80019BC85E08093380142DC8091E1003C
:1016400084FF2EC08091E20084FF2AC080E189BD22
:1016500089B5826089BD09B400FEFDCF8091D800B4
:101660008F7D8093D8008091E1008F7E8093E10090
:101670008091E2008F7E8093E2008091E2008160A1
:101680008093E20080913601882331F48091E30059
:1016900087FD02C081E001C084E08093380114DC42
:1016A0008091E10083FF22C08091E20083FF1EC091
:1016B0008091E100877F8093E10082E08093380190
:1016C000109236018091E1008E7F8093E10080913D
:1016D000E2008E7F8093E2008091E200806180933F
:1016E000E20080E060E042E350DE95D1FF91EF91AF
:1016F000BF91AF919F918F917F916F915F914F912A
:101700003F912F910F900FBE0F901F9018950F9340
:101710001F93DF93CF93CDB7DEB7AC970FB6F89496
:10172000DEBF0FBECDBF8091F10080933901809163
:10173000F10080933A018091F1009091F100EBE388
:10174000F1E080933B0190933C018091F1009091F6
:10175000F10080933D0193838091F1009091F1001D
:1017600080933F019583B3DB8091E80083FF3AC10A
:101770008091390130913A01353009F487C0363013
:1017800040F43130C9F1313070F0333009F02AC102
:1017900033C0383009F4F8C0393009F407C13630A5
:1017A00009F020C199C0803821F0823809F01AC1AF
:1017B00008C09091340180913501882399F092609E
:1017C00011C080913D0187708093E9008091EB000A
:1017D00090E025E0969587952A95E1F7982F9170EE
:1017E0001092E9008091E800877F8093E800909351
:1017F000F1001092F100D3C0882319F0823009F073
:10180000F1C090E08F719070009721F0029709F07D
:10181000E9C00CC080913B01813009F0E3C0109217
:101820003501333069F5809335012AC080913B0141
:10183000882331F520913D01277009F4D3C020930E
:10184000E9008091EB0080FF1BC0333021F48091D0
:10185000EB00806213C08091EB0080618093EB000D
:1018600081E090E002C0880F991F2A95E2F78093EB
:10187000EA001092EA008091EB0088608093EB0010
:101880001092E9008091E800877F8CC0882309F0DE
:10189000A9C010913B011F770FB7F8948091E80021
:1018A000877F8093E800A6DD8091E80080FFFCCF71
:1018B0008091E3008078812B8093E3008091E300A6
:1018C00080688093E300112311F482E001C083E07B
:1018D000809338010FBF86C08058823008F082C0E4
:1018E00080913B0190913C0123E08C3D920709F0EF
:1018F00033C083E08C838AE28B837FB7F894DE0168
:1019000015966EE040E050E011E2E62FF0E0109313
:101910005700849140FF03C082958F706F5F8F7076
:10192000282F30E08A3018F0C901C79602C0C901DB
:10193000C0968D939D934F5F5F4F4431510529F7BA
:101940007FBF8091E800877F8093E800CE010396F7
:101950006AE270E061D012C060913D01AE014F5F5C
:101960005F4FB4DCBC01009709F43CC08091E800F3
:10197000877F8093E80089819A81B4D08091E800C4
:101980008B778093E8002EC0803861F58091E80065
:10199000877F8093E800809136018093F1008091E9
:1019A000E8008E778093E80025DD1CC08823D1F401
:1019B00090913B019230B0F48091E800877F809352
:1019C000E8009093360116DD80913601882331F4CA
:1019D0008091E30087FD02C081E001C084E0809334
:1019E00038017BDB8091E80083FF0AC08091EB0027
:1019F00080628093EB008091E800877F8093E8000D
:101A0000AC960FB6F894DEBF0FBECDBFCF91DF917D
:101A10001F910F91089508959C0140913F015091AD
:101A200040014617570718F4F90190E045C06115C9
:101A3000710511F0AB01F8CF8091E8008E778093AB
:101A4000E80040E050E0F0CF80913801882309F4AD
:101A500045C0853009F444C08091E80083FF02C08E
:101A600081E008958091E80082FD32C08091E80015
:101A700080FF22C08091F3009091F200782F60E007
:101A8000292F30E0262B372B07C081918093F1005E
:101A9000415050402F5F3F4F4115510519F0203400
:101AA000310598F390E02034310509F491E08091FC
:101AB000E8008E778093E8004115510529F69923B7
:101AC00019F606C080913801882341F0853041F035
:101AD0008091E80082FFF6CF80E0089582E00895CB
:101AE00083E008959C0140913F01509140014617C9
:101AF000570718F4F90190E046C06115710511F01F
:101B0000AB01F8CF8091E8008E778093E80040E049
:101B100050E0F0CF80913801882309F447C0853028
:101B200009F446C08091E80083FF02C081E0089577
:101B30008091E80082FD34C08091E80080FF23C0DE
:101B40008091F3009091F200782F60E0292F30E02F
:101B5000262B372B08C084918093F1003196415099
:101B600050402F5F3F4F4115510519F0203431058A
:101B700090F390E02034310509F491E08091E80081
:101B80008E778093E8004115510521F6992309F0DD
:101B9000C1CF06C080913801882341F0853041F0E3
:101BA0008091E80082FFF6CF80E0089582E00895FA
:101BB00083E00895BF92CF92DF92EF92FF920F934E
:101BC0001F93CF93DF93182F092F7B016A0133DC1A
:101BD000B82E8823B1F5812F902F9C01E901C11403
:101BE000D10439F0F60180819181E81AF90AC80F11
:101BF000D91F00E010E022C08091E80085FD16C0EA
:101C00008091E8008B778093E800C114D10449F0FB
:101C1000F60180819181800F911F9183808385E0FF
:101C200011C06CD008DC882349F00CC08091F10011
:101C300089930894E108F1080F5F1F4FE114F10444
:101C4000D9F68B2DDF91CF911F910F91FF90EF90DF
:101C5000DF90CF90BF900895BF92CF92DF92EF9226
:101C6000FF920F931F93CF93DF93182F092F7B01C0
:101C70006A01E1DBB82E8823B1F5812F902F9C01FA
:101C8000E901C114D10439F0F60180819181E81A8B
:101C9000F90AC80FD91F00E010E022C08091E800C7
:101CA00085FD16C08091E8008E778093E800C1140E
:101CB000D10449F0F60180819181800F911F9183B9
:101CC000808385E011C01AD0B6DB882349F00CC0B0
:101CD00089918093F1000894E108F1080F5F1F4F8C
:101CE000E114F104D9F68B2DDF91CF911F910F9163
:101CF000FF90EF90DF90CF90BF9008951F93809159
:101D00003801882361F01091E9001092E900809178
:101D1000E80083FF01C0FBDC17701093E9001F91FE
:061D20000895F894FFCFC6
:101D260001FFFF8080808041FFFF0401212602041D
:041D360000000000A9
:00000001FF
